:0300000002237464
:0C237400787FE4F6D8FD75816D0223BB74
:1028F6003F065B4F666D7D077F6F0008040C020A7A
:0A290600060E0109050D030B070F73
:102483006028800930304750524D432C3030303073
:1024930030302C562C2C2C2C2C2C2C303030303033
:1024A300302C2C2C412A30300A0000004180FE3CA5
:10296E00EF75F00A84FEEF75F00A84EEC454F0FEA3
:03297E0025F0FF42
:012981002233
:10278B00E4FBFD7FD0122562E4FF12275DE4F53EEA
:10279B007416253EF582E43481F583E0FF12275D44
:0C27AB00053EE53EC3940740E7122910EC
:0127B70022FF
:0C29BB009080E3E0FDE4FFFE12292A22D8
:0A29D200AD077F107E0012292A22B3
:0A29DC00AD077F207E0012292A2299
:1028D900EFC4540F90290093FEEF540F93FF7D042A
:0C28E9007804088002C333D8FCFF2EFFE7
:0128F50022C0
:10285700300F07EFC4540FFC8004EF540FFC301007
:102867000AEC9028F693FF1228D922EC9028F693C9
:01287700FF61
:01287800223D
:10287900AB07E4FD7F9012256240107FAC12275D03
:102889007F0912275D1229107F00221229107F016A
:01289900221C
:1027B8008F3EAB3EE4FD7F9012256240177FEE12FC
:1027C800275D1229107427253EF582E43481F583AC
:0A27D800E4F0FF221229107F012215
:1020F500AF8DEFFEAD8B7C00E42DF53FEC3EF53E5C
:10210500908104E0FEA3E0FFE4FDFBFA7901F812FB
:1021150019EFA804A905AA06AB07AE3EAF3FE4FC3C
:10212500FD1219E2E41217749080FA121A7A90805F
:10213500FA121A627B007A247974784912166A9029
:1021450080FA121A7A9080FA121A627B007A407924
:102155001C784612166A9080FA121A7AE4FFFEFD80
:10216500FC9080FA121A6E12170760449080FA12DA
:102175001A6EE4FFFE7D807C3F12166A1217B2903C
:1021850080F8EEF0A3EFF09080F8E0FAA3E0FB7C96
:10219500007D64FFAE021218BF908103EFF07C0052
:1021A5007D64AF03AE021218BF908106EDF0C32225
:0121B500D356
:0121B6002206
:10250500300758C2073009289080E97444F0A37455
:1025150020F0E4A3F0A3F0A37408F0A3EFF0A374F4
:10252500FFF0A3F0A3F0E4A3F0A3F0753E0B801039
:102535009080E97402F0A37423F0A3EFF0753E03D5
:102545007B017A8079E9A209920FC210AD3E12246F
:0C255500005004D207C322D207D322C3D7
:012561002257
:102633001229109080E2E0FF2401F582E43480F552
:1026430083E004F074012FF582E43480F583E0D352
:102653009404401E9080E2E0FF2427F582E4348155
:10266300F5837401F074312FF582E43480F58374BB
:0326730001F02251
:100026001225AA12202D920BD207D20CD20DC21481
:10003600C20575100175118175120C7513017514C1
:10004600817515097F207E001229598F24E524D356
:10005600940840089080E87408F080069080E8E5EF
:1000660024F0E49080E2F09080E8E0FF9080E2E007
:10007600C39F5035E0FF2427F582E43481F583746D
:1000860001F01228799080E2E0FE2431F582E43412
:1000960080F583EFF074012EF582E43480F583EF6A
:1000A600F09080E2E004F080BE7817E62402F524A2
:0700B600E52478176670F9DC
:1000BD00D293300211C202908108E0600914F0E081
:1000CD007004C2A8D207300506A2B292968005A28E
:1000DD00B2B39296904000E044C0F538908102E0B2
:1000ED006538600DAF381225055006908102E53850
:1000FD00F09080FEE0FF7817E6C39F5003020241A7
:10010D00E4F69080E2E0FF9408502A74272FF582E0
:10011D00E43481F583E0701D9080E2E02427F582C0
:10012D00E43481F5837401F074312FF582E4348069
:10013D00F5837401F09080E2E004F09080E8E0FF38
:10014D009080E2E0C39F4008E4F0908102E0F4F07B
:10015D009080E2E0FF2431F582E43480F583E060A5
:10016D00211228799080E2E0FE2431F582E434807A
:10017D00F583EFF074012EF582E43480F583EFF012
:10018D0080589080E2E0FF2401F582E43480F5830D
:10019D00E0B4020D74312FF582E43480F5837401DF
:1001AD00F09080E2E0FF1227B8BF01129080E2E0EC
:1001BD002401F582E43480F583E004F0801C908006
:1001CD00E2E0FF2427F582E43481F583E4F0740145
:1001DD002FF582E43480F583E4F0C28EC2AAE49058
:1001ED008104F0A3F0F58DF58B9081077464F0C256
:1001FD00037817E62402F538C20875B80C7817E6AF
:10020D00FFB53804D208800330B3F2EF2402F5387D
:10021D00E5387817667004D208800320B3F2200801
:10022D000AD28ED2ABC28BD2AA8009E4908103F0A0
:10023D00908106F0E4FBFD7FD0122562500302048D
:10024D006CE4FF12275D122910E4FB7D017FD012B3
:10025D0025625003020467C20F12272B908116EFFF
:10026D00F0547F6006200C0302041F753801C20F85
:10027D0012272B74162538F582E43481F583EFF0BF
:10028D002014090538E538C3940F40E2D20F122728
:10029D002B122910300D167F107E001229598F2434
:1002AD00E52430E004C2098002D209C20D90811606
:1002BD00E030E71D20141AE4FBFD7FD0122562E427
:1002CD00FF12275D908116E0547FFF12275D1229E2
:1002DD001030140302044B300C1EC20CE4FFFE124E
:1002ED0029599080E3EFF07E007C0E7D101218AD41
:1002FD00908114EEF0A3EFF0908118E0FF54F0F52B
:10030D002BC4540FF52B75F00AA4F52BEF540F25C4
:10031D002BF52B90811AE0FF54F0F528C4540FF5FE
:10032D002875F00AA4F528EF540F2528F528A3E029
:10033D00FF54F0F527C4540FF52775F00AA4F527DF
:10034D00EF540F2527F527A3E0FF54F0F53AC454D9
:10035D000FF53A75F00AA4F53AEF540F253AF53A30
:10036D0024D0F526E43407F525908117E0FF54F0ED
:10037D00F52AC4540FF52A75F00AA4F52AEF540F87
:10038D00252AF52AE4F529F52C752D00752E25F570
:10039D002F753000753129852F41853042853143C8
:1003AD00AB2CAA2DA92E1222E78F358E348D338CCE
:1003BD00322093089081257401F08005E490812509
:1003CD00F0AF35AE34AD33AC32852F458530468533
:1003DD003147908125E0F548AB2CAA2DA92E121C92
:1003ED006FAF2B12296E9080D5EFF0AF2812296ECA
:1003FD009080D7EFF0AF2712296EA3EFF0E52624FA
:10040D0030FF12296EA3EFF0908117E09080D4F0A9
:10041D00802CD20F12272B122910908116E030E775
:10042D001D20141AE4FBFD7FD0122562E4FF122774
:10043D005D908116E0547FFF12275D122910908187
:10044D0016E0547FFF908000E06F6016D20AE490B2
:10045D008113F0908000EFF08008122910800312B4
:10046D0029109080E2E0FB2427F582E43481F583A6
:06047D00E06003020660CE
:10048300FD7F90122562500302065D7FAC12275D4B
:10049300920E9080E2E0FB7D017F90122562500373
:1004A30002065D7F0A1229C7D20F12272B8F24530E
:1004B3002480E52470030206589080E2E0FBE4FD0B
:1004C3007F90122562500302065D7FAA12275D907A
:1004D30080E2E0FB7D017F90122562500302065DFE
:1004E300C20F12272B9080E2E025E024BFF582E4BF
:1004F3003480F583EFF0D20F12272B9080E2E0FED9
:1005030025E024C0F582E43480F583EFF074272ED0
:10051300F582E43481F5837401F02007030205DCDE
:10052300C207300968EE25E024BFF582E43480F584
:1005330083E0753C00F53D30E70BE4253DF53D7464
:10054300FF353CF53CE53D25E0F53DE53C33F53C29
:100553009080E2E025E024C0F582E43480F583E076
:100563006003433D019080E97448F0A37461F0E4B3
:10057300A3F09080E2E024809080ECF0A37402F07A
:10058300A3E53DF0E53CA3F0753B0780399080E996
:100593007404F0A37421F09080E2E09080EBF025E6
:1005A300E024C0F582E43480F583E09080ECF090A1
:1005B30080E2E025E024BFF582E43480F583E09017
:1005C30080EDF0753B057B017A8079E9A209920FF2
:1005D300C210AD3B122400D2079080E2E0FF245307
:1005E300F582E43480F583E4F0EF25E024BFF5825F
:1005F300E43480F583E0FFF53B533B80E53B6055F6
:100603009080E2E0FE25E024BFF582E43480F583A8
:10061300EFF4F074532EF582E43480F5837402F022
:100623009080E2E0FF25E024C0F582E43480F58386
:10063300E05480F0EF25E024C0F582E43480F583B4
:10064300E070129080E2E025E024BFF582E434807C
:0D065300F583E004F0122910800312263315
:0306600030036AFA
:10066300C2031220F5300762C20730092A9080E9DD
:100673007448F0A37461F0E4A3F0A37488F0A37446
:1006830002F09080F9E09080EEF09080F8E09080A6
:10069300EFF0753B0780209080E97405F0A3742088
:1006A300F0A3E58BF0A3E58DF0908105E09080ED5C
:1006B300F0E4A3F0753B067B017A8079E9A2099205
:0A06C3000FC210AD3B122400D20755
:1006CD0020180302134F30910302089E9080E3E03F
:1006DD009080D4F0E4A3F0C200E47817F620900BDC
:1006ED009080D4E004F0D2003090FD20920B9080E9
:1006FD00D4E014F0D2003092FD9080D4E0C3940D7C
:10070D004002E4F020180302087FE4F524AF24052D
:10071D0024745B2FF582E43480F5837402F0AF24EA
:10072D000524745B2FF582E43480F583E4F0AF2467
:10073D000524745B2FF582E43480F5837401F0AFEA
:10074D00240524745B2FF582E43480F583740FF057
:10075D009080D5E0FFD20FD210122857AE24052479
:10076D00745B2EF582E43480F583EFF09080D4E055
:10077D00FF12296ED20FD210122857AE2405247401
:10078D005B2EF582E43480F583EFF09080D4E0FFAA
:10079D0012296EC20FC210122857AE240524745BA5
:1007AD002EF582E43480F583EFF0745B2524F58219
:1007BD00E43480F583E05480F0AF240524745B2F7E
:1007CD00F582E43480F583C083C082E0FB9080D550
:1007DD00E0FFC20FC210122857EB4FD082D083F02A
:1007ED00E4F538753901745B2539F582E43480F50B
:1007FD0083E02538F5380539E539B408E96338FF64
:10080D00E53824FD600824FA600424077011AF2434
:10081D000524745B2FF582E43480F5837409F0AF01
:10082D00240524745B2FF582E43480F583E538F0DC
:10083D00AF240524745B2FF582E43480F5837403B3
:10084D00F0AF240524745B2FF582E43480F583E446
:10085D00F0AF240524745B2FF582E43480F583E436
:10086D00F0908113F0D20A908126E524F0C2183061
:10087D0018FD2091030206E6D20C3000149080D4AE
:10088D00E0540F9080E3F09080DBF0F4A3F0122998
:10089D00BB309003020A18D20CC200E47817F62080
:1008AD00910AA209B39209D2003091FD20920AA2B9
:1008BD0009B39209D2003092FD2018030209FFE41A
:1008CD00F524AF240524745B2FF582E43480F58381
:1008DD007402F0AF240524745B2FF582E43480F5A7
:1008ED0083E4F0AF240524745B2FF582E43480F5A6
:1008FD00837401F0AF240524745B2FF582E43480FA
:10090D00F583740FF0AF240524745B2FF582E43466
:10091D0080F583E4F03009047F7A80027FCEAE2427
:10092D000524745B2EF582E43480F583EFF03009F5
:10093D00047F7380027F76AE240524745B2EF582CE
:10094D00E43480F583EFF03009047F3E80027F06AA
:10095D00AE240524745B2EF582E43480F583EFF02C
:10096D00E4F538753901745B2539F582E43480F589
:10097D0083E02538F5380539E539B408E96338FFE2
:10098D00E53824FD600824FA600424077011AF24B3
:10099D000524745B2FF582E43480F5837409F0AF80
:1009AD00240524745B2FF582E43480F583E538F05B
:1009BD00AF240524745B2FF582E43480F583740332
:1009CD00F0AF240524745B2FF582E43480F583E4C5
:1009DD00F0AF240524745B2FF582E43480F583E4B5
:1009ED00F0908113F0D20A908126E524F0C21830E0
:1009FD0018FD2090030208A8D20C30000E30090417
:100A0D007F0080027F018F241229D2309203020BC6
:100A1D009B9080E8E09080D4F0E4A3F0C200E478ED
:100A2D0017F62090139080E8E004F0E0D39408408E
:100A3D0002E4F0D2003090FD2091149080E8E01493
:100A4D00F0E0C3940050037408F0D2003091FD2003
:100A5D001803020B88E4F524AF240524745B2FF5ED
:100A6D0082E43480F5837402F0AF240524745B2F87
:100A7D00F582E43480F583E4F0AF240524745B2F14
:100A8D00F582E43480F5837401F0AF240524745BA2
:100A9D002FF582E43480F583740FF0AF24052474B0
:100AAD005B2FF582E43480F583E4F0AF24052474E4
:100ABD005B2FF582E43480F583E4F09080E8E0FF6D
:100ACD0012296EC20FC210122857AE240524745B72
:100ADD002EF582E43480F583EFF0AF240524745BAA
:100AED002FF582E43480F583E4F0F538753901741F
:100AFD005B2539F582E43480F583E02538F538053A
:100B0D0039E539B408E96338FFE53824FD60082478
:100B1D00FA600424077011AF240524745B2FF5824D
:100B2D00E43480F5837409F0AF240524745B2FF54C
:100B3D0082E43480F583E538F0AF240524745B2F0F
:100B4D00F582E43480F5837403F0AF240524745BDF
:100B5D002FF582E43480F583E4F0AF240524745B33
:100B6D002FF582E43480F583E4F0908113F0D20AFE
:100B7D00908126E524F0C2183018FD209203020A58
:100B8D002BD20C3000089080E8E0FF1229DCE4F550
:100B9D0024AF240524745B2FF582E43480F583742F
:100BAD0002F0AF240524745B2FF582E43480F583C5
:100BBD00E4F0AF240524745B2FF582E43480F583D3
:100BCD007401F0AF240524745B2FF582E43480F5B5
:100BDD0083740FF09080D5E0FFC3941050067E0013
:100BED007F008007D20FD210122857AE240524742F
:100BFD005B2EF582E43480F583EFF09080D4E0FF36
:100C0D00D20FD210122857AE240524745B2EF58214
:100C1D00E43480F583EFF09080D4E0FFC20FC21072
:100C2D00122857AE240524745B2EF582E43480F52A
:100C3D0083EFF0745B2524F582E43480F583E05472
:100C4D0080F0745B2524F582E43480F583C083C085
:100C5D0082E0FB9080D5E0FFC20FC210122857EB47
:100C6D004FD082D083F0AF240524745B2FF582E43E
:100C7D003480F583E06480F0E4F538753901745BF8
:100C8D002539F582E43480F583E02538F5380539CA
:100C9D00E539B408E96338FFE53824FD600824FA26
:100CAD00600424077011AF240524745B2FF582E4D2
:100CBD003480F5837409F0AF240524745B2FF5821D
:100CCD00E43480F583E538F0AF240524745B2FF50B
:100CDD0082E43480F5837403F0AF240524745B2F14
:100CED00F582E43480F583E4F0AF240524745B2FA2
:100CFD00F582E43480F583E4F0AF240524745B2F92
:100D0D00F582E43480F5837402F0852439AF24052F
:100D1D0024745B2FF582E43480F583E4F0AF240571
:100D2D0024745B2FF582E43480F583E4F0AF240561
:100D3D0024745B2FF582E43480F583740FF090807A
:100D4D00D7E0FFD20FD210122857AE240524745BC2
:100D5D002EF582E43480F583EFF09080D8E0FFD259
:100D6D000FD210122857AE240524745B2EF582E4A1
:100D7D003480F583EFF09080D8E0FFC20FC21012DF
:100D8D002857AE240524745B2EF582E43480F58358
:100D9D00EFF09080D7E0FFC20FC210122857EF443A
:100DAD0080FFAE240524745B2EF582E43480F58338
:100DBD00EFF0E4F538E539C395245014745B25390B
:100DCD00F582E43480F583E02538F538053980E582
:100DDD006338FFE53824FD600824FA6004240770A9
:100DED0011AF240524745B2FF582E43480F58374F0
:100DFD0009F0AF240524745B2FF582E43480F5836C
:100E0D00E538F0AF240524745B2FF582E43480F5CA
:100E1D00837403F0AF240524745B2FF582E43480D2
:100E2D00F583E4F0AF240524745B2FF582E4348060
:100E3D00F583E4F0AF240524745B2FF582E4348050
:100E4D00F5837402F0E4F539AF240524745B2FF5B6
:100E5D0082E43480F583E4F0AF240524745B2FF530
:100E6D0082E43480F5837409F0AF240524745B2F7C
:100E7D00F582E43480F5837403F02539F539AF2418
:100E8D000524745B2FF582E43480F583740FF0250F
:100E9D0039F539908031E06043AF240524745B2F20
:100EAD00F582E43480F583E4F0AF240524745B2FE0
:100EBD00F582E43480F583E4F0AF240524745B2FD0
:100ECD00F582E43480F583E4F0AF240524745B2FC0
:100EDD00F582E43480F583E4F0020FBC908053E09A
:100EED00B40211AF240524745B2FF582E43480F530
:100EFD00837409F0908053E0FFAE240524745B2EBB
:100F0D00F582E43480F583EFF0EF2539F5399080E3
:100F1D00BFE0FF12296EC20FD210122857EF440105
:100F2D00FF745B2524F582E43480F583EFF0745B68
:100F3D002524F582E43480F583E02539F53905243F
:100F4D009080C0E07017AF240524745B2FF582E408
:100F5D003480F583743FF02539F5398015AF2405BC
:100F6D0024745B2FF582E43480F583746DF025399C
:100F7D00F5399080BFE0FF12296ED20FC2101228F2
:100F8D00578F38E538B43F12AF240524745B2FF525
:100F9D0082E43480F583E4F08015AF240524745B7E
:100FAD002FF582E43480F583E538F02539F5396382
:100FBD0039FFE53924FD600824FA60042407701117
:100FCD00AF240524745B2FF582E43480F583740916
:100FDD00F0AF240524745B2FF582E43480F583E5AE
:100FED0039F0AF240524745B2FF582E43480F5834A
:100FFD007403F0AF240524745B2FF582E43480F57F
:10100D0083E4F0AF240524745B2FF582E43480F57E
:10101D0083E4F0AF240524745B2FF582E43480F56E
:10102D00837402F0E4F539AF240524745B2FF58247
:10103D00E43480F583E4F0AF240524745B2FF5824E
:10104D00E43480F5837409F0AF240524745B2FF527
:10105D0082E43480F5837402F005390539AF240537
:10106D0024745B2FF582E43480F583740FF02539F9
:10107D00F539908032E06043AF240524745B2FF581
:10108D0082E43480F583E4F0AF240524745B2FF5FE
:10109D0082E43480F583E4F0AF240524745B2FF5EE
:1010AD0082E43480F583E4F0AF240524745B2FF5DE
:1010BD0082E43480F583E4F002119B908054E0B417
:1010CD000211AF240524745B2FF582E43480F5837F
:1010DD007409F0908054E0FFAE240524745B2EF566
:1010ED0082E43480F583EFF0EF2539F5399080C136
:1010FD00E0FF12296EC20FD210122857EF4401FFE4
:10110D00745B2524F582E43480F583EFF0745B2560
:10111D0024F582E43480F583E02539F539052490F2
:10112D0080C2E07017AF240524745B2FF582E43480
:10113D0080F583743FF02539F5398015AF240524EA
:10114D00745B2FF582E43480F583746DF02539F5E9
:10115D00399080C1E0FF12296ED20FC210122857AC
:10116D008F38E538B43F12AF240524745B2FF58218
:10117D00E43480F583E4F08015AF240524745B2FEF
:10118D00F582E43480F583E538F02539F539633996
:10119D00FFE53924FD600824FA600424077011AFBF
:1011AD00240524745B2FF582E43480F5837409F0F3
:1011BD00AF240524745B2FF582E43480F583E53983
:1011CD00F0AF240524745B2FF582E43480F583742D
:1011DD0003F0AF240524745B2FF582E43480F5838E
:1011ED00E4F0AF240524745B2FF582E43480F5839D
:1011FD00E4F0AF240524745B2FF582E43480F5838D
:10120D007402F0852439AF240524745B2FF582E434
:10121D003480F583E4F0AF240524745B2FF582E46C
:10122D003480F5837404F0AF240524745B2FF582AC
:10123D00E43480F583740FF0908103E0FF12296E82
:10124D00D20FD210122857AE240524745B2EF582CE
:10125D00E43480F583EFF0908106E0FF12296ED221
:10126D000FD210122857AE240524745B2EF582E49C
:10127D003480F583EFF0908106E0FF12296EC20FE6
:10128D00C210122857AE240524745B2EF582E43467
:10129D0080F583EFF0908103E0FF12296EC20FC23B
:1012AD0010122857EF4480FFAE240524745B2EF5F1
:1012BD0082E43480F583EFF0E4F538E539C3952405
:1012CD005014745B2539F582E43480F583E02538BC
:1012DD00F538053980E56338FFE53824FD600824CD
:1012ED00FA600424077011AF240524745B2FF58276
:1012FD00E43480F5837409F0AF240524745B2FF575
:10130D0082E43480F583E538F0AF240524745B2F37
:10131D00F582E43480F5837403F0AF240524745B07
:10132D002FF582E43480F583E4F0AF240524745B5B
:10133D002FF582E43480F583E4F0C218908126E520
:10134D0024F02014030200BD30A8030200BDC21416
:10135D00E4F536F5377524029081C6E0FF24FEFED4
:10136D00E524C39E501874C72524F582E43481F515
:10137D0083E02536F5362537F537052480DA74C533
:10138D002FF582E43481F583E0653660030200BDFC
:10139D009081C6E024C6F582E43481F583E065379B
:1013AD0060030200BD9081E0E064076005C20502A4
:1013BD0000BDD2059081DFE075F00A84E5F0600391
:1013CD000200BD9081DCE0FF12296E90811AEFF0D2
:1013DD009081DBE0FF12296E90811BEFF09081DA96
:1013ED00E09081D9E024002430FF12296E90811CF9
:1013FD00EFF09081DFE0FF12296E908116EFF090F3
:10140D0081DEE0FF12296E908117EFF09081DDE013
:10141D00FF12296E908118EFF0C2AC12278BD20CFF
:10142D00D2AC2009030214FB9081DDE0F52B9081F5
:10143D00DCE0F5289081DBE0F5279081DAE0FE9085
:10144D0081D9E07C002400F526EC3EF5259081DE67
:10145D00E0F52AA3E0F529752C00752D00752E25D4
:10146D00752F00753000753129852F4185304285E6
:10147D003143AB2CAA2DA92E1222E78F358E348D38
:10148D00338C32AF35AE34AD33AC32E47B01FAF987
:10149D00F81219E28F358E348D338C32908043746F
:1014AD0001F0A37418F0A37480F0A37401F0A37479
:1014BD0006F0A3E535F0A3E534F0A3E533F0A3E59D
:1014CD0032F0E4A3F0A3F09081C6740BF020070373
:1014DD0002164FC2077A807943E0FDA209920FD21E
:1014ED0010122400400302164FD20602164F9081AF
:1014FD0018E0FD54F0FEC4540F2430908011F0ED2F
:10150D00540F2430A3F0908117E0FD54F0FEC45425
:10151D000F2430908013F0ED540F2430A3F0908100
:10152D0016E004F0E0FD54F0FEC4540F243090801A
:10153D0015F0ED540F2430A3F09080187441F09005
:10154D00811AE0FD54F0FEC4540F2430908020F039
:10155D00ED540F2430A3F090811BE0FD54F0FEC438
:10156D00540F2430908022F0ED540F2430A3F090CE
:10157D00811CE0FD54F0FEC4540F2430908024F003
:10158D00ED540F2430A3F0752401E4F539740925C9
:10159D0024F582E43480F583E0642A601274C72553
:1015AD0024F582E43481F583E06239052480DE057B
:1015BD0024E53954F0FFC4540FF538D39409501471
:1015CD00E5382430FF74092524F582E43480F58351
:1015DD00EFF08012E5382437FF74092524F582E4F5
:1015ED003480F583EFF00524E539540FF538D394A5
:1015FD00095014E5382430FF74092524F582E434AC
:10160D0080F583EFF08012E5382437FF7409252427
:10161D00F582E43480F583EFF09081C67428F030C4
:10162D000720C207E0FD14908009F0A37424F07B1D
:10163D00017A807909A209920FD21012240050026A
:10164D00D206300607C206D2070200BDC289D2A853
:06165D009081087416F0F4
:031663000200BDC5
:011666002261
:0A29C700E4FEEEC39F50030E80F8FB
:0129D10022E3
:0D29A100904001E04440F07F141229C7224D
:0D29AE00904001E054BFF07F141229C722B1
:0F2982001229A1C210309502D2101229AEA21054
:012991002223
:02275D00AD07C6
:10275F00E4FCED30E709904001E04420F080079061
:10276F004001E054DFF0122982ED25E0FD0CBC089A
:0B277F00E1904001E04420F0122982AC
:01278A00222C
:10272B00E4FDFC12298250010DED25E0FD0CBC07E8
:10273B00F212298250010D904001E054DFF0300F6E
:10274B0004E04420F0122982904001E04420F0AFD5
:01275B000578
:01275C00225A
:02256200AC07C4
:10256400EB6009904001E04480F08007904001E076
:10257400547FF01229AE904001E04420F07F141201
:1025840029C71229A1904001E054DFF07F141229D9
:10259400C71229AEE4FFEB600514FE25E0FFEC2D25
:0525A4002FFF12275D6E
:0125A900220F
:102910001229AE904001E054DFF07F141229C71253
:0A29200029A1904001E04420F022BC
:0F29920045746865726E6574206661696C21001A
:1024B300602C822DFFFFFFFFFFFFFFFFFFFFFFFFEA
:1024C300FACE000000000000000000000000000041
:1024D30000000000000000000000000000000000F9
:1024E3005E826008004500002D007B400040113AE9
:1024F3004600000000FFFFFFFF03CD03CD001900DE
:0125030000D7
:10202D00D2B47F641229C7C2B47F641229C790034A
:10203D00007421F07817E62402FF7817E6B5070241
:10204D00D322900300E0B421F190030E7448F09078
:10205D00030AE4F0A3F0A3F0A37402F0900301745B
:10206D0044F0A3744FF0A37444F090030774FFF091
:10207D0090030F7401F0900308E4F0A3F0A3742013
:10208D00F0A3E4F0900300740AF0754A01754B82D9
:10209D00754C33E4FE900310E0FD784AE475F001D1
:1020AD00121A86ED121879900310E0FF0EBE06E5A8
:1020BD009003007461F0754A01754B82754C33E4E1
:1020CD00FE784AE475F001121A8612183390030156
:1020DD00F00EBE06EC9003077444F09003007422DA
:0720ED00F090030DE4F0C3C5
:0120F40022C9
:1027E20090030AE4F0A3F09003007422F09003082F
:1027F200E4F0A37440F0EF2410FFA3F0A3E4F09000
:0828020003007422F07412F0CF
:01280A0022AB
:06289A008B488A49894ABF
:1028A000E4FFEFC39D50137848E475F001121A86D7
:0A28B000121833900310F00F80E8B7
:0128BA0022FB
:102833007548037549E8301312E5491549700215C7
:1028430048144548700512202DD322900300E02040
:03285300E2E4C3F9
:01285600225F
:101F5B008B448A4589468D47A2129213122833501F
:101F6B00012290030AE4F0A3F09003007422F09096
:101F7B000308E4F0A37440F0E547D394404007E531
:101F8B00472410FF80027F4090030AEFF0A3E4F098
:101F9B009003007422F07412F07B017A82792D7D0C
:101FAB000612289A7B017A82793312289A20111E05
:101FBB0090823974FAF0A374CEF0A3E547F0E4A352
:101FCB00F07B017A8279397D0412289A801EE547CD
:101FDB00240E90827BF07B017A8279607D1E122821
:101FEB009A7B017A8279337D0612289AAB44AA45F3
:101FFB00A946AD4712289A9003047440F0E547D3E5
:10200B0094404008E5472410A3F080069003057424
:10201B0040F0900306E4F02012069003007426F0C3
:02202B00C322CE
:06225A008B448A45894611
:10226000ED2404FF7E04EEC39F501C7844E475F017
:1022700001121A86121833FD742F2EF582E4348170
:10228000F583EDF00E80DFE4FDFCFEEF30E0107B27
:10229000000EEB242FF582E43481F583E0FD1FEE80
:1022A000C39F5022AB060E742F2BF582E43481F5C8
:1022B00083E06204AB060E742F2BF582E43481F5C3
:1022C00083E0620580D9AF060E742F2FF582E434C7
:1022D00081F583ECF0AF060E742F2FF582E4348184
:0622E000F583EDF0AF06EE
:0122E60022D5
:082400008B3F8A4089418D42A7
:10240800200F1A90812F74FFF0A3F0E4A3F0A374B7
:102418001FF012225AE5422406F543802BE4F543C7
:10242800E543C39542501E783FE475F001121A86C1
:10243800121833FF742F2543F582E43481F583EFB6
:10244800F0054380DB8542437B017A81792FA20F17
:102458009211A2109212AD43121F5B501C7BFF7A9F
:102468002979927D0F12225AAD077BFF7A2979923A
:0A247800C211C212121F5BD322C36F
:012482002237
:0729E6009003007426F022AB
:1025AA00C292D292E47817F6758911758815D28D80
:1025BA00438E0275C83C75CDFF75CBFF75CCD975B6
:1025CA00CAD9C204759850D2AFD2A9D2ACC297C2A6
:1025DA0096D218C21690822B04F01229AE78007691
:0525EA00FF1229A122EF
:030013000228BB05
:1028BB00C0E0C083C082908107E014F0E07006C2D4
:0E28CB008EC2AAD203C28BD082D083D0E0325C
:1026F7000000001F003B005A0078009700B500D487
:1027070000F301110130014E016D0000001F003C74
:10271700005B0079009800B600D500F40112013182
:04272700014F016EEF
:0621B7008B5F8A60896164
:1021BD00121960AEF0244EF563EE34F8F56290001E
:1021CD000212184C24FFF565E434FFF564E5632431
:1021DD0001FFE43562FE7C007D04121914AA06ABE2
:1021ED0007AE62AF637C017D6D1218ADEF2BFDEE76
:1021FD003AFCE56525E0FFE56433FE74F72FF582C3
:10220D0074263EF5837401932DFFE4933CFEAB5F82
:10221D00AA6090000312184C7C002FFFEC3ECF24D7
:10222D00FFCF34FFAB07FAAE62AF637D0412191412
:10223D00ED64024C7012C3E5659402E5646480940C
:0C224D008040050BBB00010AAE02AF038D
:012259002262
:0A1B64008E5F8F608B618A628963D7
:101B6E00EE3395E08F6D8E6CF56BF56AE47F04FEB7
:101B7E00FDFCAB6DAA6CA96BA86A1219EFEF2402DB
:101B8E00FFE43EFEE43DFDE43CFCE47BB57A05F962
:101B9E00F81225EF8E648F65E5652401FFE4356448
:101BAE00FE7C007D04121914AA06AB07AE64AF6565
:101BBE007C017D6D1218ADEF2BFFEE3AFEC3E56092
:101BCE009FF569E55F9EF568AE64AF651C7D0412F6
:101BDE001914ED64024C70087BFF7A277911800688
:101BEE007BFF7A2679F77D017C00ED25E0FFEC3353
:101BFE008F82F58312198BFFC3E5699FE5F0648030
:101C0E00F8E568648098400B0DBD00010CED640C86
:101C1E004C70D7ED24FFFFEC34FFFEEF25E0FFEE16
:101C2E00338F82F58312198BFFAEF0C3E5699FF5F2
:101C3E0067E5689EF566E56524B2FFE5643407AB9B
:101C4E0061AA62A9638FF01219C3AB61AA62A9637C
:101C5E00900002ED12188BE5670490000312188BAA
:011C6E002253
:10294300EF2403FFE43EFE7C007D07121914ED24FF
:0629530001FFE43CFE223E
:081D72008F4E8E4D8D4C8C4B01
:101D7A007B807A51790178001225EF8E4F8F507B44
:101D8A00007A007953121B6475550375561F7B0040
:101D9A007A0079531221B78E4F8F501229437C0053
:101DAA007D071219148C518D52C3E5509552FFE5E7
:101DBA004F9551FE3395E0FDFC7B807A517901788D
:101DCA00001219EFEF2420F55AEE341CF559E43DC0
:101DDA00F558E43CF55775550A75561F7B007A008D
:101DEA0079531221B78E4F8F501229437C007D07F9
:101DFA001219148C518D52C3E5509552FFE54F9537
:101E0A0051FE3395E0FDFC7B807A5179017800120E
:101E1A0019EFEF2420F55EEE341CF55DE43DF55C28
:101E2A00E43CF55BAF5AAE59AD58AC57AB4EAA4D30
:101E3A00A94CA84BC3121A4C5004E4FEFF22AF5E11
:101E4A00AE5DAD5CAC5BAB4EAA4DA94CA84BC312C0
:0C1E5A001A4C4004E4FEFF227E007F01D1
:011E66002259
:0E1C6F008F418E408D3F8C3E8B428A438944CC
:101C7D00908114E0FEA3E0FFE4FCFDE5412FF5416A
:101C8D00E5403EF540ED353FF53FEC353EF53EE5A3
:101C9D00486025AF41AE40AD3FAC3E121D72EF4ED8
:101CAD006016E5412410F541E540340EF540E4356C
:101CBD003FF53FE4353EF53EE54445434542601C66
:101CCD007B807A5179017800AF41AE40AD3FAC3E9B
:101CDD001225EFAB42AA43A944121B64E5474546C2
:101CED0045457003021D71AF41AE40AD3FAC3E7B2B
:101CFD00807A51790178001225EFAC00AD01AE026A
:101D0D00AF038F418E408D3F8C3EE47B107A0EF9F0
:101D1D00F81225EFAB45AA46A947900002EF12181D
:101D2D008BE47B107A0EF9F8AF41AE40AD3FAC3E7F
:101D3D001225EFAE02AF038E498F4A7C007D3C1217
:101D4D001914AB45AA46A947900001EF12188BAEA6
:101D5D0049AF4A7C007D3C121914AB45AA46A947F0
:041D6D00ED121879E2
:011D7100224F
:1022E7001221B7EE3395E0FDFC7B807A51790178B6
:1022F700001219EFC004C005C006C007AB41AA42CF
:10230700A94390000212184CFFE4FCFDFE7B107AF3
:102317000EF9F81219EFD003D002D001D00012192C
:10232700E2C004C005C006C007AB41AA42A943905A
:10233700000112184CFFE4FCFDFE7B3CFAF9F81291
:1023470019EFD003D002D001D0001219E2A804C0BF
:1023570005C006C007AB41AA42A943121833FFE4E0
:0C236700FCFDFED003D002D0011219E2F0
:012373002247
:03000B0002267654
:10267600C0E0C083C082C0D075D008C28D758AAF55
:10268600758C3CD2B5908113E004F0E0640A6003D7
:10269600300A0AC20A201905201802D299D20278F5
:1026A6001706E67002F5A8C2B5D0D0D082D083D086
:0226B600E03210
:03001B0002280BAD
:10280B00C0E0C0F0C083C082C0D075D000C000C291
:10281B008F908104E475F00112194AD000D0D0D00A
:08282B0082D083D0F0D0E0322E
:03002300021E6753
:0B1E6700C0E0C083C082C0D075D0185E
:101E7200209803021F14C298301403021F52301616
:101E82002D9081C6E024C7F582E43481F583E5997B
:101E9200F09081C6E004F09081C5E0FFA3E0C39F0B
:101EA2005003021F52C216C297D214021F52301799
:101EB2004C9081C6E024C7F582E43481F583E5992C
:101EC200F09081C6E004F0E0FFC394075003021FC4
:101ED20052C2179081C8E0646270759081C9E06453
:101EE20001706D9081CAE064217065D2169081CB39
:101EF200E02F547F9081C5F0E004F08053E599B45F
:101F0200B510D2979081C7E599F09081C67401F01F
:101F1200D21730993BC2993019230516908126E0D9
:101F2200FFE516C39F5010745B2516F582E43480DA
:101F3200F583E0F5998019C219D2188013D2197568
:101F42001600745B2516F582E43480F583E0F5997A
:091F5200D0D0D082D083D0E0325F
:030003000226B81A
:1026B800C0E0C0F0C083C082C0D075D000C000C0E8
:1026C80001C002C003C004C005C006C0071229E645
:1026D800D207C2A8D007D006D005D004D003D002B4
:0F26E800D001D000D0D0D082D083D0F0D0E0325B
:10295900438E2075D2028F828E83E0FFE4F5D25335
:042969008EDFD2AF7C
:01296D002247
:10292A00E5D220E0FBC2AF43D2028F828E83EDF064
:09293A0075D25075D2A0D2AF2273
:10166700021828EC5D046005E85904700302181E8F
:101677001217E9580460F6EC4860F2EC7004FDFEBE
:10168700FF22C860DB2481C85009C3986002500656
:101697000218259850CAF582E9294B4A7005AB8292
:1016A70002181475F0007C1A7880C3EF9BEE9AED50
:1016B70099400DC3EF9BFFEE9AFEED99FDE842F0CE
:1016C700DC23ACF0D0E0FFD0E0FED0E0FDAB822021
:1016D700E7101BEB60BAEC2CFCEF33FFEE33FEEDAB
:1016E70033FD021800E803F830E705C0F075F00095
:1016F700EF2FFFEE33FEED33FD40B830E7C280AA8F
:1017070074F8CC6480CCC86480C8F582046043C395
:10171700EB9FF5F0EA9E42F0E99D42F0E89C45F028
:1017270060305018E5825FFFE582F42B5582FB504D
:10173700210ABA001D09B90019088016E5825BFB6A
:10174700E582F42F5582FF50090EBE00050DBD003E
:10175700010CC3EB9FF5F0EA9E42F0E99D42F0E8E9
:0D1767009C45F06007CC4820E701B3EC2260
:1017740075F020800E75F010800575F0087D007EF0
:10178400007F003392D530D503121A3EEC3340105B
:10179400EF33FFEE33FEED33FDEC33FCD5F0ED22F9
:0E17A400E5F0247EA2D513CC92E7CDCEFF2235
:1017B200EDD2E7CD33EC3392D524814006E4FFFE2F
:1017C200FDFC22FCE4CFCECDCC24E0501174FF808E
:1017D200EDC3CC13CCCD13CDCE13CECF13CF04702B
:0717E200F030D5DE021A3ED3
:1017E900E9D2E7C933E833F892D5EDD2E7CD33EC46
:0717F90033FC5002B2D522BF
:10180000EC30E7100FBF000C0EBE00080DBD000449
:101810000BEB6014A2D5EB13FCED92E7FD2274FFF5
:10182000FCFDFEFF22E480F8A2D574FF13FC7D804E
:03183000E480EF62
:10238000020026E493A3F8E493A34003F68001F24D
:1023900008DFF48029E493A3F85407240CC8C3335E
:1023A000C4540F4420C8834004F456800146F6DF2D
:1023B000E4800B0102040810204080902483E47E16
:1023C000019360BCA3FF543F30E509541FFEE49322
:1023D000A360010ECF54C025E060A840B8E493A3E9
:1023E000FAE493A3F8E493A3C8C582C8CAC583CA14
:1023F000F0A3C8C582C8CAC583CADFE9DEE780BECC
:0125040000D6
:10183300BB010689828A83E0225002E722BBFE02B3
:09184300E32289828A83E49322E6
:10184C00BB010CE58229F582E5833AF583E0225051
:10185C0006E92582F8E622BBFE06E92582F8E2229B
:0D186C00E58229F582E5833AF583E49322B5
:10187900BB010689828A83F0225002F722BBFE014E
:02188900F32248
:10188B00F8BB010DE58229F582E5833AF583E8F093
:10189B00225006E92582C8F622BBFE05E92582C83F
:0218AB00F22227
:1018AD00EF8DF0A4A8F0CF8CF0A428CE8DF0A42E4F
:0218BD00FE2209
:1018BF00BC000BBE0029EF8DF084FFADF022E4CC0D
:1018CF00F875F008EF2FFFEE33FEEC33FCEE9DECD6
:1018DF00984005FCEE9DFE0FD5F0E9E4CEFD22ED1C
:1018EF00F8F5F0EE8420D21CFEADF075F008EF2F66
:1018FF00FFED33FD4007985006D5F0F222C398FD57
:05190F000FD5F0EA22F3
:10191400C2D5EC30E709B2D5E4C39DFDE49CFCEEEE
:1019240030E715B2D5E4C39FFFE49EFE1218BFC38F
:10193400E49DFDE49CFC80031218BF30D507C3E48A
:061944009FFFE49EFE225D
:10194A00C5F0F8A3E028F0C5F0F8E5821582700228
:06195A001583E038F022C5
:10196000BB010A89828A83E0F5F0A3E02250068752
:10197000F009E71922BBFE07E3F5F009E319228914
:0B198000828A83E493F5F07401932247
:10198B00BB0110E58229F582E5833AF583E0F5F09A
:10199B00A3E0225009E92582F886F008E622BBFE77
:1019AB000AE92582F8E2F5F008E222E5832AF583BD
:0819BB00E993F5F0A3E9932282
:1019C300BB010A89828A83F0E5F0A3F0225006F76F
:0F19D30009A7F01922BBFE06F3E5F009F319226C
:0D19E200EF2BFFEE3AFEED39FDEC38FC2254
:1019EF00E88FF0A4CC8BF0A42CFCE98EF0A42CFC97
:1019FF008AF0EDA42CFCEA8EF0A4CDA8F08BF0A415
:101A0F002DCC3825F0FDE98FF0A42CCD35F0FCEB73
:101A1F008EF0A4FEA9F0EB8FF0A4CFC5F02ECD3938
:0F1A2F00FEE43CFCEAA42DCE35F0FDE43CFC22A5
:1025EF00C2D5E830E70FB2D5E4C39BFBE49AFAE417
:1025FF0099F9E498F8EC30E717B2D5122625121A9C
:10260F00D2E4C39BFBE49AFAE499F9E498F88003C7
:10261F00121AD230D50DE4C39FFFE49EFEE49DFD58
:04262F00E49CFC2209
:0E1A3E00C3E49FFFE49EFEE49DFDE49CFC22B9
:101A4C00EB9FF5F0EA9E42F0E99D42F0EC6480C811
:061A5C0064809845F022B1
:0C1A6200E0FCA3E0FDA3E0FEA3E0FF22F7
:0C1A6E00E0F8A3E0F9A3E0FAA3E0FB22FB
:0C1A7A00ECF0A3EDF0A3EEF0A3EFF022DF
:101A8600FAE6FB0808E6F925F0F618E6CA3AF62261
:101A960075F008758200EF2FFFEE33FECD33CDCC07
:101AA60033CCC58233C5829BED9AEC99E58298408A
:101AB6000CF582EE9BFEED9AFDEC99FC0FD5F0D667
:101AC600E4CEFBE4CDFAE4CCF9A88222B800C1B991
:101AD6000059BA002DEC8BF084CFCECDFCE5F0CBCF
:101AE600F97818EF2FFFEE33FEED33FDEC33FCEB08
:101AF60033FB10D703994004EB99FB0FD8E5E4F9C3
:101B0600FA227818EF2FFFEE33FEED33FDEC33FCAF
:101B1600C933C910D7059BE99A4007EC9BFCE99AA3
:101B2600F90FD8E0E4C9FAE4CCFB2275F010EF2FE8
:101B3600FFEE33FEED33FDCC33CCC833C810D707E8
:101B46009BEC9AE899400AED9BFDEC9AFCE899F823
:0E1B56000FD5F0DAE4CDFBE4CCFAE4C8F922B6
:00000001FF
